:020000040800F2
:1000000000060020A102000845110008491100085F
:10001000A11100084911000875110008A302000889
:10002000A3020008A3020008A3020008A12A0008F6
:10003000A3020008A3020008A3020008A30200080C
:10004000A3020008A3020008A3020008A3020008FC
:10005000A3020008A30200084D3F0008793F0008F2
:10006000A53F0008D13F0008FD3F0008A30200089B
:10007000A3020008A3020008A3020008A3020008CC
:10008000A3020008A3020008A3020008A3020008BC
:10009000A3020008A3020008A302000829400008E8
:1000A000A3020008A3020008A3020008A30200089C
:1000B00015410008A3020008A3020008A3020008DB
:1000C000A3020008A3020008A3020008A30200087C
:1000D000A3020008A3020008A3020008A30200086C
:1000E0008D400008A3020008A3020008A302000834
:1000F000A3020008A3020008A3020008A30200084C
:10010000A3020008A3020008A3020008A30200083B
:10011000A3020008A3020008A3020008A30200082B
:10012000A3020008A3020008A3020008A30200081B
:10013000A3020008A3020008A3020008A30200080B
:10014000A3020008A3020008A3020008A3020008FB
:10015000A3020008A3020008A3020008A3020008EB
:10016000A3020008A3020008A3020008A3020008DB
:10017000A302000845360008A3020008A3020008F5
:10018000A3020008A302000801410008A30200081E
:10019000A3020008A3020008A3020008A3020008AB
:1001A000A3020008A3020008A3020008A30200089B
:1001B000A3020008A3020008A3020008A30200088B
:1001C000A3020008A3020008A3020008A30200087B
:1001D000A302000831360008A3020008A3020008A9
:1001E000A3020008A3020008A3020008A30200085B
:1001F000A3020008A3020008A3020008A30200084B
:10020000A3020008A3020008A3020008A30200083A
:10021000A3020008A3020008A3020008A30200082A
:10022000A3020008A3020008A3020008A30200081A
:10023000A3020008A3020008A3020008A30200080A
:10024000A3020008A3020008A3020008A3020008FA
:10025000A3020008A3020008A3020008A3020008EA
:10026000A3020008A3020008A3020008A3020008DA
:10027000A3020008A3020008A3020008A3020008CA
:10028000A3020008A3020008A3020008A3020008BA
:10029000A3020008A3020008A3020008A3020008AA
:1002A00002E000F000F8FEE772B63A4880F30888F2
:1002B000394880F3098839484EF60851CEF20001DA
:1002C000086040F20000CCF200004EF63471CEF22D
:1002D00000010860BFF34F8FBFF36F8F40F2000043
:1002E000C0F2F0004EF68851CEF200010860BFF374
:1002F0004F8FBFF36F8F4FF00000E1EE100A4EF604
:100300003C71CEF200010860062080F31488BFF330
:100310006F8F02F087FC02F027FC03F0D7FB4FF051
:1003200055301F491B4A91423CBF41F8040BFAE784
:100330001C49194A91423CBF41F8040BFAE71A499B
:100340001A4A1B4B9A423EBF51F8040B42F8040B69
:10035000F8E700201749184A91423CBF41F8040BC6
:10036000FAE702F045FC03F031FC144C144DAC42AA
:1003700003DA54F8041B8847F9E700F0CFF8114C72
:10038000114DAC4203DA54F8041B8847F9E702F038
:100390002DBC000000060020002200200000000804
:1003A0000000002000060020084500080022002070
:1003B0005C22002060220020F8460020A0020008F5
:1003C000A0020008A0020008A00200082DE9F04FDA
:1003D0002DED108AC1F80CD0D0F80CD0BDEC108AED
:1003E000BDE8F08F002383F311882846A047002042
:1003F00001F050FFFEE701F0D1FE00DFFEE7000054
:10040000032A70B422D940EA01039B0711D0037874
:100410000C78A3421DD10A44013105E010F8013FD8
:1004200011F8014BA34214D19142F7D1002070BCC6
:1004300070470D680668AE420C46034601F10401A0
:1004400000F1040008D1043A032AF2D8002ADED1D0
:10045000ECE7181B70BC704721461846D7E700BF71
:1004600080EA0102844612F0030F4FD111F0030F0E
:1004700032D14DF8044D11F0040F51F8043B0BD06C
:10048000A3F101329A4312F0803F04BF4CF8043BC1
:1004900051F8043B16D100BF51F8044BA3F10132CF
:1004A0009A4312F0803FA4F101320BD14CF8043B87
:1004B000A24312F0803F04BF51F8043B4CF8044BB8
:1004C000EAD023460CF8013B13F0FF0F4FEA332329
:1004D000F8D15DF8044B704711F0010F06D011F808
:1004E000012B0CF8012B002A08BF704711F0020FF6
:1004F000BFD031F8022B12F0FF0F16BF2CF8022BE1
:100500008CF8002012F47F4FB3D1704711F8012B03
:100510000CF8012B002AF9D1704700BF38B500F064
:1005200003FD30B1164B00220E211A725A729972D5
:10053000DA7202F077FA044602F0ACFA0546D0B956
:10054000104B9C4219D001339C4241F2883412BFB7
:10055000054600240125002002F06EFA0DB100F0DE
:100560005BF800F095FD00F027FC204600F014F940
:1005700000F052F8F9E70024EDE70446EBE700BF8E
:1005800000220020010007B008B500F0E1FBA0F157
:1005900020035842584108BD054B07B51B8802216E
:1005A00001A8ADF8043000F0F1FB03B05DF804FBE6
:1005B000B841000810B5202383F311881248C3689E
:1005C0000BB101F0EFFE0023104A4FF47A710E4890
:1005D00001F0AAFE002383F311880D4C236813B1A8
:1005E0002368013B2360636813B16368013B636068
:1005F000084B1B7833B9636823B9022000F0B0FCC4
:100600003223636010BD00BF60220020B5050008E2
:100610007C23002074220020554B56492DE9F041DF
:1006200053F8042F013201D1BDE8F0818B42F7D19C
:10063000514C524B22689A4240F29880504B9B6832
:1006400003F1006303F500339A4280F08F800020AD
:1006500000F0CEFB02204B4B187000F073FC4A4BAD
:10066000D3F8E8200022C3F8E820D3F81011C3F82B
:100670001021D3F81011D3F8EC10C3F8EC20D3F804
:100680001411C3F81421D3F81411D3F8F010C3F8DF
:10069000F020D3F81811C3F81821D3F81811D3F8A3
:1006A000801041F00061C3F88010D3F8801021F071
:1006B0000061C3F88010D3F88010D3F8801041F0A7
:1006C0000071C3F88010D3F8801021F00071C3F8D6
:1006D0008010D3F8803072B62C4B2D490B601D680A
:1006E0002468BFF34F8FBFF36F8F2A4BC3F884206A
:1006F000BFF34F8F5A6922F480325A61BFF34F8F94
:10070000D3F8802043F6E07EC2F3C906C2F34E322E
:10071000B707520102EA0E0838463146013948EA65
:10072000000C00F14040B1F1FF3FC3F874C2F5D1B5
:10073000203A12F1200FEDD1BFF34F8FBFF36F8F2F
:10074000BFF34F8FBFF36F8F5A6922F400325A61A3
:100750000022C3F85022BFF34F8FBFF36F8F2023C7
:1007600083F31188AD4685F308882047BDE8F08102
:10077000FCFF01081C00020804000208FFFF01083A
:1007800000220020742200200044025800000208C9
:1007900008ED00E000ED00E02DE9F04F99B0BB4D11
:1007A0002022FF21009010A8AC6800F013FCB84A8A
:1007B00001951378A3B90121B6481170C3602023B5
:1007C00083F31188C3680BB101F0ECFD0023B24A3A
:1007D0004FF47A71AF4801F0A7FD002383F311882D
:1007E000009BAE4A03B113600026AD4B009DB2469C
:1007F0003746B1461E7056600293012000F0A2FBFE
:10080000002D00F02B82A54B1B68002B40F02682A8
:1008100019B0BDE8F08F0220FFF7B6FE002840F0C7
:100820001682009B02210BA8002E08BF1D469D4B7F
:100830001B88ADF82C3000F0A9FADEE74FF47A708F
:1008400000F086FAB0F10008EBDB0220FFF79CFE17
:100850000028E6D008F1FF38B8F1050F00F2F98161
:10086000DFE808F0030B0E11143718A80523042144
:1008700040F8343D00F08AFA17E004218348F9E794
:1008800004218948F6E704218848F3E74FF01C0962
:10089000484609F1040900F0ADFA04210B900BA8B9
:1008A00000F074FAB9F12C0FF2D101234FF00009D6
:1008B00003FA08F848EA0A0A5FFA8AFA00F0DEFB4F
:1008C00027B10AF00B030B2B08BF0025FFF764FECE
:1008D00093E704217648CDE7002FA2D00AF00B035E
:1008E0000B2B9ED10220FFF74FFE8046002898D0A8
:1008F00001206B4E00F07CFA00270220307000F0DF
:1009000021FB5FFA87FB584600F082FA054688B162
:100910005846013700F08CFA0028F2D146460025EF
:10092000644B02210BA847461B88ADF82C3000F021
:100930002DFA62E701232C460220337000F0F6FA0C
:10094000019B9B689C4206D2204600F053FA01307E
:10095000E4D10434F4E70024029B464647461C7069
:1009600025464E4B5C60A9E7002F3FF45AAF0AF0D2
:100970000B030B2B7FF455AF0220029B187000F085
:10098000E1FA322000F0E4F9B0F1000BFFF649AFD4
:100990001BF003087FF445AF019B04EB0B02996841
:1009A0008A423FF63EAFBBF5807F3FF63AAF424A00
:1009B000D84503920FDA4FF47A7000F0C9F9049029
:1009C00004990029FFF62DAF0499039A08F8021044
:1009D00008F10108ECE7C820FFF7D6FD80460028A3
:1009E0003FF41FAF1F2C11D8C4F1200710AB24F027
:1009F000030031495F45184428BF5F463A4600F07E
:100A0000C1FA3A46FF212C4800F0E4FA4FEAAB0362
:100A100029492046DAB2039300F0E4FA0746002899
:100A20003FF47EAF039B04EB830447E70220FFF70C
:100A3000ABFD00283FF4F5AE00F014FA00283FF4B7
:100A4000F0AE4FF000084346019A9268904535D2C7
:100A5000B8F11F0F12D8109A01320FD028F00302FC
:100A600018A90A4452F8202C0B92184604220BA90C
:100A700008F1040800F0A8FB0346E5E740460393AD
:100A800000F0B8F9039B0B90EFE700BF00220020B5
:100A90007823002060220020B50500087C23002078
:100AA00074220020BA4100080422002008220020FD
:100AB0000C220020BC4100087822002018A8042144
:100AC00040F84C3D00F062F9F8E618A800236421D4
:100AD00040F8343D00F050F900287FF4A2AE022027
:100AE000FFF752FD00283FF49CAE0B9800F0B2F9DE
:100AF00018AB43F8480D04211846E3E718A8002373
:100B0000642140F8343D00F037F900287FF489AEC5
:100B10000220FFF739FD00283FF483AE0B9800F068
:100B20009BF918AB43F8440DE5E70220FFF72CFDD5
:100B300000283FF476AE00F0A5F918AB43F8400D5D
:100B4000D9E70220FFF720FD00283FF46AAE0BA989
:100B5000142000F09DF9804618A8042140F83C8D2F
:100B600000F014F941460BA8ACE7322000F0F0F891
:100B7000B0F10008FFF655AE18F0030F7FF451AE48
:100B8000019A08EB0903926893423FF64AAE0220AD
:100B9000FFF7FAFC00283FF444AE28F00308C844ED
:100BA000C1453FF48BAE484609F1040900F022F933
:100BB00004210A900AA800F0E9F8F1E74FF47A70EE
:100BC000FFF7E2FC00283FF42CAE00F04BF90028C0
:100BD00042D0109B01330BD0082210A9002000F056
:100BE00001FA002838D02022FF2110A800F0F2F9E5
:100BF000FFF7D2FC3A4801F053FB09E6002F3FF41F
:100C000010AE0AF00B030B2B7FF40BAE18A80023D9
:100C1000642140F8343D00F0AFF8804600287FF4AE
:100C200000AE0220FFF7B0FC00283FF4FAAD0390BD
:100C3000FFF7B2FC41F28830454601F031FB0B98DA
:100C400000F060FA00F01AFA039B1F46D5E507464C
:100C500034E64FF00009E4E5B84661E6002000F014
:100C600077F80490049B002BFFF6CAAD012000F03A
:100C70005DF9049B213B162B3FF6BFAD01A252F854
:100C800023F000BF170800083D080008D908000835
:100C9000FB070008FB070008FB07000869090008BC
:100CA0006B0B00082D0A0008CB0A0008FD0A00089B
:100CB0002B0B0008FB070008430B0008FB0700088C
:100CC000BD0B0008BD080008FB070008FD0B00086D
:100CD00023080008BD080008FB070008CB0A00082D
:100CE000A08601002DE9F84F4FF47A7507460E46AD
:100CF00000245543DFF85080DFF8509098F9003019
:100D00005FFA84FA5A1C01D0A34210D159F824008A
:100D1000324639460368D3F820B02B46D84786427E
:100D200005D1084B012083F800A0BDE8F88F0134FD
:100D3000022CE3D14FF4FA7001F0B2FA0020BDE8C2
:100D4000F88F00BFC823002010220020C0410008F7
:100D500007B5002202AB012103F8012D0246184617
:100D6000FFF7C0FF20B19DF8070003B05DF804FB5A
:100D70004FF0FF30F9E700000A46042108B5FFF7FD
:100D8000B1FF80F00100C0B2404208BD074B30B453
:100D90001A78074B53F822400A460146236820463A
:100DA000DD69044BAC4630BC604700BFC82300205F
:100DB000C0410008A0860100F8B50A4C00250A4E83
:100DC00001F016FD094F208030682388834207D93F
:100DD00001F00AFD336805440133BD423360F3D9A5
:100DE000F8BD00BFCA23002084230020FFFF0100BC
:100DF00001F0CCBD00F1006000F5003000687047E4
:100E000000F10060920000F5003001F04DBD0000DF
:100E1000054B1A68054B1B889B1A834202D9104464
:100E200001F0E2BC0020704784230020CA23002088
:100E300038B5074D04462868204401F0DBFC28B98A
:100E400028682044BDE8384001F0E6BC38BD00BF4A
:100E50008423002000207047014BC058704700BF1A
:100E600000E8F11F064991F8243033B1002308222D
:100E7000086A81F82430FFF7C3BF0120704700BF24
:100E800088230020014B1868704700BF0010005CE9
:100E9000234BF0B5234C1B682788C3F30B0665680A
:100EA0001B0C94F90820BE4228D0A789BE4206D167
:100EB00001220C2505FB0244656894F9082041F2E3
:100EC0000104A3421CD041F20304A3421AD042F20F
:100ED0000104A34218D042F20304A34208BF5622E1
:100EE000441E013D0B460C44A34217D215F9016F75
:100EF000581C5EB1034600F8016CF5E70022D8E704
:100F00005A22EDE75922EBE75822E9E72C258442E3
:100F10001D7001D9981C5A70401AF0BD1846FBE7A5
:100F20000010005C1422002000207047022803D12A
:100F30000422034B9A6170470128FCD10222F8E792
:100F400000100258022804D14FF48022034B9A610A
:100F500070470128FCD14FF40032F7E70010025827
:100F6000022805D1064A536983F004035361704790
:100F70000128FCD1024A536983F00203F6E700BF5F
:100F800000100258002310B5934203D0CC5CC45427
:100F90000133F9E710BD000030B5441E14F9010F0C
:100FA0000B4658B193F900500131854206D11AB968
:100FB00093F90020801A30BD013AEFE7002AF7D1FB
:100FC000104630BD02460346981A13F9011B00294A
:100FD000FAD1704702440346934202D003F8011B42
:100FE000FAE770472DE9F047234C05468846174637
:100FF00094F8243083BB2E46DFF87C90C7B394F876
:1010000024302BB92022FF2148462662FFF7E2FF59
:1010100094F824004146C0F1080504EB8000BD426D
:1010200028BF3D465FFA85FAAD00A7EB0A072A46BE
:101030002E44FFF7A7FF94F82430A844FFB29A4447
:101040005FFA8AFABAF1080F84F824A0D6D1FFF724
:1010500009FF0028D2D108E0266A06EB8306B042D9
:10106000CAD0FFF7FFFE0028C5D10020BDE8F087F9
:101070000120BDE8F08700BF88230020024B1A78CA
:10108000024B1A70704700BFC823002010220020B6
:1010900038B5164C164D204600F000FC2946204677
:1010A00000F028FC2D681348D5F89020D2F80438B9
:1010B00043F00203C2F8043801F0F2F80E49284662
:1010C00000F02AFDD5F890200C48D2F804380C49DD
:1010D000A04223F00203C2F804384FF4E1330B605E
:1010E00003D0BDE8384000F037BB38BDF029002000
:1010F000C842000840420F00F0420008CC23002004
:10110000B023002038B50B4B05461A780A4B53F82C
:1011100022400A4B9C420CD0094B00211822184651
:10112000FFF758FF056001462046BDE8384000F053
:1011300013BB38BDC8230020C0410008F02900209F
:10114000B0230020FEE7000000B59BB0EFF309815B
:1011500068226846FFF716FFEFF30583044B9A6B8E
:10116000DA6A9A6A9A6A9A6A9A6A9A6A9B6AFEE73D
:1011700000ED00E000B59BB0EFF3098168226846FE
:10118000FFF700FFEFF30583044B9A6B9A6A9A6AA4
:101190009A6A9A6A9A6A9B6AFEE700BF00ED00E0CD
:1011A00000B59BB0EFF3098168226846FFF7EAFEBD
:1011B000EFF30583034B5A6B9A6A9A6A9A6A9A6AA2
:1011C0009B6AFEE700ED00E030B50A44074D91420E
:1011D0000BD011F8013B09245840013CF7D040F3F3
:1011E00000032B4083EA5000F7E730BD2083B8EDC1
:1011F000026843681143016003B11847704700005B
:10120000024A136843F0C00313607047007800403F
:1012100013B50E4C204600F093FA04F1140000942C
:1012200000234FF400720A4900F054F90094094B6E
:101230004FF40072084904F1380000F0CDF9074B73
:10124000E365074B236602B010BD00BFCC2300202E
:1012500038240020011200083826002000780040C1
:1012600000E1F505254B002908BF1946037C012B39
:1012700030B511D1224B98420ED1224BD3F8E82041
:1012800042F08042C3F8E820D3F8102142F08042B7
:10129000C3F81021D3F810310A68036EC46D03EB54
:1012A00052038166B3FBF2F34A68150442BF23F090
:1012B000070503F0070343EA4503E3608B6843F047
:1012C00040036360CB68510543F00103A36042F41F
:1012D000967343F0010323604FF0FF33236205D57B
:1012E00012F0102205D0B2F1805F04D080F8643093
:1012F00030BD7F23FAE73F23F8E700BFE441000851
:10130000CC230020004402582DE9F047C66D054665
:101310003768F469200734621AD014F0080F0CBF44
:1013200000218021E20748BF41F02001A3074FF0D0
:10133000200348BF41F04001600748BF41F480717D
:1013400083F31188281DFFF753FF002383F31188CF
:10135000E2050AD5202383F311884FF40071281D7C
:10136000FFF746FF002383F311884FF020094FF069
:10137000000A14F0200831D13B0616D54FF02009A1
:1013800005F1380A200610D589F31188504600F07F
:1013900057F900282FDA0821281DFFF729FF27F029
:1013A00080033360002383F3118879060DD562062C
:1013B0000BD5202383F31188EA6C2B6D9A4201D15F
:1013C0002B6CEBB9002383F31188E30620D5AA6EBA
:1013D0001369EBB15069BDE8F047184789F31188EC
:1013E000736A284695F86410194000F0C3F98AF32F
:1013F0001188F469BDE7B06288F31188F469C1E728
:1014000027F040071021281DFFF7F2FE3760D9E7CB
:10141000BDE8F087F8B51546826804460B46AA4237
:1014200000D28568A1692669761AB54207D21846A6
:101430002A46FFF7A7FDA3692B44A3610DE011D94C
:10144000AF1B32461846FFF79DFD3A46E16830442F
:10145000FFF798FDE2683A44A261A36828465B1B47
:10146000A360F8BD18462A46FFF78CFDE368E4E761
:10147000836893422DE9F04104460F46154600D299
:10148000856860692669361AB54207D22A46394608
:10149000FFF778FD63692B4463610EE013D9A5EB78
:1014A000060832463946FFF76DFD4246B919E06835
:1014B000FFF768FDE26842446261A36828465B1B4F
:1014C000A360BDE8F0812A463946FFF75BFDE3687B
:1014D000E2E7000010B50A440024C361029B0060EB
:1014E00040608460C160816141610261036210BD3E
:1014F00008B582694369934201D1826882B98268E2
:10150000013282605A1C42611970426903699A4231
:1015100001D3C3684361002100F0DEFE002008BD56
:101520004FF0FF3008BD000070B5202304460E4682
:1015300083F31188A568A5B1A368A269013BA360E4
:10154000531CA36115782269934224BFE368A36109
:10155000E3690BB120469847002383F3118828469E
:1015600070BD3146204600F0A7FE0028E2DA85F380
:10157000118870BD2DE9F74F05460F4690469A46F3
:10158000D0F81C90202686F311884FF0000B1446EB
:1015900064B1224639462846FFF73CFF034668B946
:1015A0005146284600F088FE0028F1D0002383F33E
:1015B0001188A8EB040003B0BDE8F08FB9F1000F6B
:1015C00003D001902846C847019B8BF31188E41A89
:1015D0001F4486F31188DBE7C160816141611144DA
:1015E000C361009B006040608260016103627047DC
:1015F000F8B504460E461746202383F31188A568E4
:10160000A5B1A368013BA36063695A1C62611E70A7
:10161000236962699A4224BFE3686361E3690BB19D
:1016200020469847002080F31188F8BD39462046AF
:1016300000F042FE0028E2DA85F31188F8BD0000D0
:10164000836942699A4210B501D182687AB9826889
:10165000013282605A1C82611C7803699A4201D36C
:10166000C3688361002100F037FE204610BD4FF0B3
:10167000FF3010BD2DE9F74F05460F4690469A46BC
:10168000D0F81C90202686F311884FF0000B1446EA
:1016900064B1224639462846FFF7EAFE034668B998
:1016A0005146284600F008FE0028F1D0002383F3BD
:1016B0001188A8EB040003B0BDE8F08FB9F1000F6A
:1016C00003D001902846C847019B8BF31188E41A88
:1016D0001F4486F31188DBE7026843681143016009
:1016E00003B11847704700001430FFF743BF0000F4
:1016F0004FF0FF331430FFF73DBF00003830FFF7E5
:10170000B9BF00004FF0FF333830FFF7B3BF000020
:101710001430FFF709BF00004FF0FF311430FFF71E
:1017200003BF00003830FFF763BF00004FF0FF3207
:101730003830FFF75DBF000000207047FFF768BD3D
:10174000044B0360002343608360C3600123037480
:10175000704700BFFC41000810B52023044683F306
:101760001188FFF77FFD02232374002383F3118880
:1017700010BD000038B5C36904460D461BB90421ED
:101780000844FFF7A9FF294604F11400FFF7B0FE53
:10179000002806DA201D4FF48061BDE83840FFF7CD
:1017A0009BBF38BD026843681143016003B118470D
:1017B0007047000037B5446B41F6A40563591A68B9
:1017C0001178042914D1217C022911D1197901231E
:1017D00012898B4013420BD101A904F14C0002F095
:1017E00079F864590246019B2179206800F0ECF9F0
:1017F00003B030BD143001F0FDBF00004FF0FF33E7
:10180000143001F0F7BF00004C3002F0CFB80000F8
:101810004FF0FF334C3002F0C9B80000143001F033
:10182000CBBF00004FF0FF31143001F0C5BF000006
:101830004C3002F09BB800004FF0FF324C3002F009
:1018400095B8000070B541F6A406054682591368A4
:101850001978042901D0012070BD017C0229FAD138
:10186000527901205C8990400440F4D105F11400C4
:1018700001F05CFF02460028EDD0AD594FF44073F3
:101880002868697900F08EF9204670BD406BFFF73B
:10189000D9BF000000207047704700007FB5124B91
:1018A00001250426044603600023057400F1840228
:1018B000436029468360C3600C4B0290143001934F
:1018C0004FF44073009601F00DFF094B04F694426B
:1018D0002946019304F14C004FF4407302940096A2
:1018E00001F0D4FF04B070BD244200088D18000838
:1018F000B51700080A68202383F311880B790B338E
:1019000042F823004B79133342F823008B7913B14B
:101910000B3342F8230041F6A403C15002230374A1
:10192000002383F31188704738B5037F044613B151
:1019300090F85430ABB90125201D0221FFF732FF8A
:1019400004F1140025776FF0010100F0D1FC84F858
:10195000545004F14C006FF00101BDE8384000F034
:10196000C7BC38BD10B5012104460430FFF71AFF8B
:101970000023237784F8543010BD000038B50446A6
:101980000025143001F0C6FE04F14C00257701F06B
:1019900095FF201D84F854500121FFF703FF2046D6
:1019A000BDE83840FFF74EBF90F8803003F0600389
:1019B000202B19D190F88120212A0AD0222A4FF019
:1019C00000030ED0202A0FD1084A426707228267FF
:1019D00004E0064B4367072383670023C3670120A6
:1019E000704743678367F9E7002070472C22002087
:1019F00073B541F6A405044643591A6811780429C1
:101A000019D1017C022916D11979012312898B4041
:101A1000134210D100F14C06304602F00FF850B1DD
:101A200001A9304601F056FF64590246019B217915
:101A3000206800F0C9F802B070BD000001F10B038E
:101A4000F7B550F8234005460E46F4B1202383F342
:101A5000118805EB8607201D08214C34FFF7A2FEF4
:101A6000FB685B691B6813B1204601F041FF01A9C7
:101A7000204601F02FFF024648B1019B314628461F
:101A800000F0A2F8002383F3118803B0F0BDFB68D7
:101A90005A691268002AF5D01B8A013B1340F1D124
:101AA00005F18002EAE70000133138B550F8214013
:101AB000E4B1202383F3118841F6A403E2581368AC
:101AC000527903EB8203DB689B695D6845B10421B1
:101AD0006018FFF767FE294604F1140001F030FE9C
:101AE0002046FFF7AFFE002383F3118838BD0000C6
:101AF0007047000001F012B9012300F1300200F13B
:101B0000500103700023436042F8043B8A42D361D2
:101B1000FAD103814381704738B50446202383F30B
:101B20001188002500F10C0300F13002416043F8F8
:101B3000045B9342FBD1204601F012F9022323708B
:101B400085F3118838BD000070B500EB81030546B0
:101B500050690E461446DA6018B110220021FFF7D2
:101B600039FAA06918B110220021FFF733FA314683
:101B70002846BDE8704001F005BA0000038900F175
:101B80003002002103F001030381438903F00103C4
:101B9000438100F1100343F8041B9342FBD101F091
:101BA00089BA0000F0B4012500EB810447898D401B
:101BB000E4683D43A469458123600023A26063601B
:101BC000F0BC01F0A5BA0000F0B4012500EB8104DF
:101BD00007898D40E4683D436469058123600023E3
:101BE000A2606360F0BC01F01DBB0000022300F1A5
:101BF0000C0200F1300110B5037004460023A0F878
:101C0000883080F88A3080F88B300381438142F835
:101C1000043B8A42FBD184F87030204601F046F93B
:101C200063681B6823B120460021BDE810401847B7
:101C300010BD0000037880F88C30052303704368E2
:101C40001B6810B504460BB104219847002323817B
:101C5000638110BD436890F88C201B6802700BB143
:101C6000052118477047000090F8703070B50446A1
:101C700013B1002380F8703004F18002204601F097
:101C80003DFA63689B6863BB94F8805015F060066A
:101C900015D194F8813005F07F0545EA032540F21F
:101CA00002339D4200F00E815BD8022D00F0DC80F3
:101CB0003FD8002D00F08780012D00F0CF8000215B
:101CC000204601F0D5FC0021204601F0C5FC6368E8
:101CD0001B6813B1062120469847062384F870300C
:101CE00070BD204698470028CED094F8872094F8FD
:101CF000863043EA0223A26F934238BFA36794F968
:101D00008030A56F002B4FF0200380F2FD80002D66
:101D100000F0EC80092284F8702083F31188002100
:101D2000A36F626F2046FFF74FFF002383F31188F4
:101D300070BDB5F5817F00F0B180B5F5407F49D029
:101D4000B5F5807FBBD194F88230012BB7D1B4F8C0
:101D5000883023F00203A4F888306667A667E66738
:101D6000C3E740F201639D421ED8B5F5C06F3BD278
:101D7000B5F5A06FA3D1B4F88030B3F5A06F0ED144
:101D800094F88230204684F88A3001F0EDF86368D8
:101D90001B6813B1012120469847032323700023B9
:101DA0006367A367E367A0E7B5F5106F32D040F62D
:101DB00002439D4252D0B5F5006F80D104F18B03F0
:101DC0006367012324E004F18803E5676367022366
:101DD000A3678AE794F88230012B7FF470AFB4F8E0
:101DE000883043F00203B6E794F885202046616806
:101DF00094F884304D6843EA022394F8831094F8F1
:101E00008220A84700283FF45AAF436863670368FD
:101E1000A367A4E72378042B10D1202383F3118830
:101E20002046FFF7ABFE86F311886368032184F830
:101E30008B601B6821700BB12046984794F8823064
:101E4000002BACD084F88B300423237063681B68AC
:101E5000002BA4D0022120469847A0E7374B6367A8
:101E60000223A36700239DE794F88410204611F015
:101E7000800F01F00F010ED001F032F9012806D0D9
:101E800002287FF41CAF2E4BA067636767E72D4BDA
:101E9000A567636763E701F015F9EFE794F882300F
:101EA000002B7FF40CAF94F8843013F00F013FF453
:101EB00076AF1A06204602D501F0F2FB6FE701F07B
:101EC000E3FB6CE794F88230002B7FF4F8AE94F8D3
:101ED000843013F00F013FF462AF1B06204602D599
:101EE00001F0C6FB5BE701F0B7FB58E7142284F86A
:101EF000702083F311882B462A4629462046FFF797
:101F000051FE85F3118870BD5DB1152284F87020F3
:101F100083F311880021A36F626F2046FFF742FE12
:101F200003E70B2284F8702083F311882B462A469E
:101F300029462046FFF748FEE3E700BF5442000869
:101F40004C4200085042000838B590F87030044602
:101F5000152B29D8DFE803F03E28282828283E281A
:101F6000280B293928282828282828283E3E90F898
:101F7000871090F88620836F42EA01229A4214D992
:101F8000C268128AB3FBF2F502FB15356DB9202346
:101F900083F311882B462A462946FFF715FE85F361
:101FA00011880A2384F8703038BD142384F8703007
:101FB000202383F31188002320461A461946FFF791
:101FC000F1FD002383F3118838BDC36F03B1984737
:101FD0000023E7E7002101F04BFB0021204601F040
:101FE0003BFB63681B6813B1062120469847062314
:101FF000D8E7000090F87020152A38B5044622D89A
:102000000123934040F6416213421DD113F4801521
:102010000FD19B0217D50B2380F87030202383F358
:1020200011882B462A462946FFF7CEFD85F31188F5
:1020300038BDC3689B695B682BB9C36F03B1984710
:10204000002384F8703038BD002101F011FB00211D
:10205000204601F001FB63681B6813B1062120468E
:1020600098470623EDE70000024B00221B605B60EF
:102070009A60704738280020002382680374054B5B
:102080001B6899689142FBD25A68036042601060F5
:10209000586070473828002008B5202383F3118842
:1020A000037C032B05D0042B0DD02BB983F31188AF
:1020B00008BD436900221A604FF0FF334361FFF708
:1020C000DBFF0023F2E790E80C001A60026853601F
:1020D000F2E70000002382680374054B1B689968CF
:1020E0009142FBD85A6803604260106058607047A4
:1020F00038280020054B1969087418680268536075
:102100001A60186101230374FEF760B938280020B3
:102110004B1C30B5054687B00A4C10D0236901A886
:10212000094A00F001F92846FFF7E4FF049B13B1C8
:1021300001A800F037F92369586907B030BDFFF7EF
:10214000D9FFF8E7382800209920000838B50C4D51
:10215000044641612B6981689A68914203D8BDE8C1
:102160003840FFF789BF1846FFF7B4FF01232C6101
:10217000014623742046BDE83840FEF727B900BF6A
:1021800038280020044B1A681B6990689B689842A5
:1021900094BF0020012070473828002010B5084C5B
:1021A000236820691A6854602260012223611A742E
:1021B000FFF790FF01462069BDE81040FEF706B921
:1021C00038280020FEE7000010B50C4CFFF74CFF4C
:1021D00000F09CF880220A49204600F021F80123F3
:1021E00044F8180C037400F06BFC002383F311888F
:1021F00062B60448BDE8104000F034B86028002002
:10220000584200086042000800F008B9034B5968C2
:102210005A68521A9042FBD8704700BF001000E085
:102220008260022202740022427470478368A3F124
:102230007C0243F80C2C026943F83C2C426943F8B9
:10224000382C074A43F81C2CC268A3F1180043F845
:10225000102C022203F8082C002203F8072C7047E8
:10226000E503000810B5202383F31188FFF7DEFF94
:1022700000210446FFF76AFF002383F311882046FC
:1022800010BD0000024B1B6958610F20FFF732BFE1
:1022900038280020202383F31188FFF7F3BF0000C4
:1022A00008B50146202383F311880820FFF730FF8B
:1022B000002383F3118808BD49B1064B42681B69AE
:1022C00018605A60136043600420FFF721BF4FF08D
:1022D000FF307047382800200368984206D01A68FB
:1022E0000260506018465961FFF7C6BE7047000093
:1022F00038B504460D462068844200D138BD0368D5
:1023000023605C604561FFF7B7FEF4E7054B03F11E
:1023100014025A619A614FF0FF32DA6100221A62A8
:10232000704700BF38280020F8B503610E46C26030
:10233000054601F0B7FB1A4B19461F4651F8142FFA
:102340008A420DD118620A2E2CBF80190A30AE6065
:102350006A602A609D615D61BDE8F84001F090BB54
:102360001B6A9268C41A341928BF3446A24202D9A3
:10237000181901F093FB7B699A6894420CD8AC6001
:1023800098685A68041B2B606A6015605D609C60E9
:102390004FF0FF33FB61F8BDA41A1B68ECE700BFE8
:1023A0003828002038B51C4B01685A691D469042F8
:1023B0000DD044682160002102685460C1609168BA
:1023C0008068014491604FF0FF32DA6138BD1A46EF
:1023D00042F8141F4A6000215B69C160934203D137
:1023E000BDE8384001F054BB9A6881680A449A609D
:1023F0002C6A01F057FB6A69001B926882420AD975
:10240000111A092998BF00F10A02286ABDE838406C
:10241000104401F043BB38BD382800202DE9F041BD
:10242000184D002705F114066C6901F03BFB2A6A80
:10243000A368811A8B4216D81344D4F80C802B62FF
:1024400094E80C001A60226853606B69E760B3423D
:1024500001D101F01DFB87F311882069C0472023BB
:1024600083F31188E0E76A69B24208D05B1ABDE8DD
:10247000F0410A2B2CBFC0180A3001F00FBBBDE899
:10248000F08100BF3828002000207047FEE70000E0
:10249000704700004FF0FF3070470000022906D05F
:1024A000032906D00129064818BF002070470548B7
:1024B0007047032A9ABF044800EBC200002070470F
:1024C0004C430008004300083C22002070B59AB03D
:1024D00006460846144601AD294600F0BDF82846D8
:1024E000FEF770FDC0B2431C5B0086E81800237045
:1024F0000323023404F8013C00231946DAB2023403
:10250000904201D81AB070BDEA5C013304F8011C96
:1025100004F8022CF2E7000008B5202383F31188A9
:102520000348FFF765FA002383F3118808BD00BF55
:10253000F029002090F8803003F01F02012A07D113
:1025400090F881200B2A03D100234367836712E0B0
:1025500003F06003202B11D1B0F8843073B990F8E8
:102560008120212A03D0222AEFD0202A06D1044A32
:10257000426707228267C36701207047FFF714BADA
:102580003322002010B50446052916D8DFE801F0F3
:1025900016150316161D202383F311880E4A0121F8
:1025A000FFF7D2FA20460D4A0221FFF7CDFA0C4878
:1025B000FFF7E4F9002383F3118810BD202383F390
:1025C00011880748FFF7B0F9F4E7202383F3118857
:1025D0000348FFF7C7F9EDE780420008A44200086E
:1025E000F029002038B50C4D0C4C2A460C4904F15A
:1025F0000800FFF76BFF05F1CA0204F1100009495A
:10260000FFF764FF05F5CA7204F118000649BDE83A
:102610003840FFF75BBF00BFC84200203C220020CB
:10262000D0420008DA420008E542000870B50446CE
:1026300008460D46FEF7C6FCC6B2204601340378B4
:102640000BB9184670BD32462946FEF7A5FC002896
:10265000F3D1012070BD00002DE9F04704460D467E
:10266000FEF7B0FC2A49C6B22046FFF7DFFF08B1EB
:102670000936F6B227492046FFF7D8FF08B11036D1
:10268000F6B2632E0BD8DFF88880DFF88890224FEF
:10269000DFF890A0267846B92E70BDE8F087214675
:1026A0002846BDE8F047FDF7DBBE252E2CD10722DA
:1026B00041462046FEF770FC60B9184B2A4603F1EC
:1026C000100153F8040B8B4242F8040BF9D1073484
:1026D0001035DFE7082249462046FEF75DFC98B931
:1026E000AA1C0F4B13F8011F023209095345C95D9B
:1026F00002F8041C197801F00F01C95D02F8031CEF
:10270000F0D118350834C5E72E7001340135C1E722
:102710006C430008E5420008854300087443000844
:10272000FFE7F11F0BE8F11FBFF34F8F044B1A694E
:102730005107FCD1D3F810215207F8D1704700BFE0
:102740000020005208B50D4B1B78ABB9FFF7ECFF2A
:102750000B4BDA68D10704D50A4A5A6002F1883275
:102760005A60D3F80C21D20706D5064AC3F80421D3
:1027700002F18832C3F8042108BD00BF26450020BD
:10278000002000522301674508B5114B1B78F3B9AF
:10279000104B1A69510703D5DA6842F04002DA603B
:1027A000D3F81021520705D5D3F80C2142F040028E
:1027B000C3F80C21FFF7B8FF064BDA6842F00102BC
:1027C000DA60D3F80C2142F00102C3F80C2108BDF5
:1027D00026450020002000520F289ABF00F5806097
:1027E00040040020704700004FF4003070470000A4
:1027F000102070470F2808B50BD8FFF7EDFF00F544
:1028000000330268013204D104308342F9D101203F
:1028100008BD002008BD00000F2810B504463FD8B1
:10282000FFF782FFFFF78EFF1E484FF0FF33072CA4
:102830004361C0F814311DD80361FFF775FF23020F
:1028400043F02403C360C36843F08003C36003699B
:102850005A07FCD4FFF768FF2046FFF7BDFF4FF48F
:10286000003100F0F9F8FFF78FFF2046BDE8104077
:10287000FFF7C0BFC0F81031FFF756FFA4F10803FF
:102880001B0243F02403C0F80C31D0F80C3143F0A4
:102890008003C0F80C31D0F810315B07FBD4D9E7C6
:1028A000002010BD002000522DE9F84F40EA02033D
:1028B000054689469046DB065AD122F003020346BC
:1028C0000244934205D1FFF73DFF4E46DFF8B8B012
:1028D00042E0196801314BD10433F2E7264A05F191
:1028E000784326489342264B264F88BF9A46A3F149
:1028F000FC039CBFDA46184603F1F80388BF1F4665
:10290000FFF712FF4FF0FF3306F11C02A5EB060E96
:1029100003603B6843F002033B60331FDAF800407A
:1029200014F00504FAD153F8041F9A424EF803102C
:10293000F4D1BFF34F8FFFF7F7FE4FF0FF332022A4
:102940003146036028463B6823F002033B60FDF7F5
:1029500057FD58B920352036A8EB06034B441F2BF2
:10296000BCD80120FFF710FFBDE8F88F2046F9E73B
:102970000020BDE8F88F00BFFFFF0F0014210052B8
:10298000102100520C2000521020005210B5084CAB
:10299000237828B153B9FFF7D5FE0123237010BD6A
:1029A00023B12070BDE81040FFF7EEBE10BD00BFA0
:1029B0002645002002440439064BD2B210B590429D
:1029C00000D110BD441C00B253F8200041F8040FA0
:1029D000E0B2F4E7504000580F4B30B51C6F2404B0
:1029E00005D41C6F1C671C6F44F400441C670B4C1F
:1029F000024404392368D2B243F480732360084B45
:102A0000904200D130BD441C51F8045F00B243F83D
:102A10002050E0B2F4E700BF0044025800480258DA
:102A20005040005807B5012201A90020FFF7C2FF5E
:102A3000019803B05DF804FB13B50446FFF7F2FFFD
:102A4000A04206D002A90122002041F8044DFFF760
:102A5000C3FF02B010BD00000144BFF34F8F064B0F
:102A6000884204D3BFF34F8FBFF36F8F7047C3F813
:102A70005C022030F4E700BF00ED00E0034B1B6870
:102A80005B0142BF0122024B1A707047D0440258CA
:102A900027450020014B1878704700BF27450020CC
:102AA000EFF30983054968334A6822F001024A605E
:102AB00083F30988002383F31188704730EF00E027
:102AC000202080F3118862B60D4B0E4AD96821F49C
:102AD000E0610904090C0A430B49DA60CA6842F054
:102AE0008072CA60094A0A49C2F8B01F116841F0F1
:102AF000010111601022DA7783F82200704700BFCD
:102B000000ED00E00003FA05F0ED00E0001000E049
:102B100055CEACC510B5202383F311880E4B5B68EE
:102B200013F4006314D0F1EE103AEFF309844FF080
:102B30008073683CE361094BDB68236684F3098892
:102B4000FFF720FB10B1064BA36110BD054BFBE75F
:102B500083F3118810BD00BF00ED00E030EF00E00E
:102B6000F7030008FA030008F0B5BFF34F8FBFF377
:102B70006F8F1D4B0021C3F85012BFF34F8FBFF36F
:102B80006F8F5A6942F400325A61BFF34F8FBFF31F
:102B90006F8FC3F88410BFF34F8FD3F8802043F6B4
:102BA000E076C2F3C904C2F34E32A507520102EA2D
:102BB000060E284621464EEA0007013900F1404042
:102BC000C3F860724F1CF6D1203A12F1200FEED1FB
:102BD000BFF34F8F5A6942F480325A61BFF34F8F6F
:102BE000BFF36F8FF0BD00BF00ED00E0FEE7000017
:102BF000084A094B09498B4204D3094A00219342F0
:102C000005D3704752F8040F43F8040BF3E743F879
:102C1000041BF4E760450008F8460020F846002051
:102C2000F846002070470000D0F89430002170B5BD
:102C3000D0F890404FF0FF359E684A01A318D3F8B2
:102C40000009002805DAD3F8000940F08040C3F8F5
:102C50000009D3F8000B002805DAD3F8000B40F088
:102C60008040C3F8000B0131A3188E42C3F8085905
:102C7000C3F8085BE1D24FF00113C4F81C3870BDF3
:102C800000EB81032DE9F04FD3F80CE04F1C4FEA25
:102C90004118DEF814403F03D4F800C06568D0F84E
:102CA000902065450AD30120D2F8343800FA01F1AA
:102CB00023EA0101C2F83418BDE8F08FACEB05033C
:102CC000BEF81060B34228BF334602EB0806D6F8C0
:102CD0001869B6B2B3EB860F13D8A6683A44994682
:102CE000A6F1040A5AF804BFB9F1040FC2F800B003
:102CF00002D9A9F10409F5E71E442B44A6606360DC
:102D0000CCE70020BDE8F08F890141F0200101618E
:102D100003699B06FCD41220FFF778BA10B50A4C61
:102D20002046FEF7E9FE094BC4F89030084BC4F882
:102D30009430084C2046FEF7DFFE074BC4F8903075
:102D4000064BC4F8943010BD284500200000084010
:102D5000BC430008C445002000000440C8430008EC
:102D60000378012B70B505465DD1494BD0F89040F2
:102D7000984259D1474B0E216520D3F8D82042F014
:102D80000062C3F8D820D3F8002142F00062C3F8F3
:102D90000021D3F80021D3F8802042F00062C3F86C
:102DA0008020D3F8802022F00062C3F88020D3F87E
:102DB000803000F081FC384BE360384BC4F80038B9
:102DC0000023D5F89060C4F8003EC02323604FF480
:102DD0000413A3633369002BFCDA01230C20336155
:102DE000FFF714FA3369DB07FCD41220FFF70EFA61
:102DF0003369002BFCDA00262846A660FFF714FF93
:102E00006B68C4F81068DB68C4F81468C4F81C6800
:102E1000002B3AD1224BA3614FF0FF336361A368CB
:102E200043F00103A36070BD1E4B9842C8D1194BFB
:102E30000E214D20D3F8D82042F00072C3F8D820DC
:102E4000D3F8002142F00072C3F80021D3F800212A
:102E5000D3F8802042F00072C3F88020D3F880209D
:102E600022F00072C3F88020D3F88020D3F8D82055
:102E700022F08062C3F8D820D3F8002122F08062CB
:102E8000C3F80021D3F8003193E7074BC3E700BF35
:102E9000284500200044025840140040030020024E
:102EA000003C30C0C4450020083C30C0F8B5D0F824
:102EB0009040054600214FF000662046FFF724FFB2
:102EC000D5F8941000234FF001128F684FF0FF30B7
:102ED000C4F83438C4F81C2804EB431201339F4271
:102EE000C2F80069C2F8006BC2F80809C2F8080B02
:102EF000F2D20B68D5F89020C5F8983063621023A1
:102F00001361166916F01006FBD11220FFF77EF947
:102F1000D4F8003823F4FE63C4F80038A36943F4FE
:102F2000402343F01003A3610923C4F81038C4F808
:102F300014380B4BEB604FF0C043C4F8103B094B07
:102F4000C4F8003BC4F81069C4F80039D5F89830CB
:102F500003F1100243F48013C5F89820A362F8BD72
:102F60009843000840800010D0F8902090F88A1014
:102F7000D2F8003823F4FE6343EA0113C2F80038A4
:102F8000704700002DE9F0410EB20D4600EB8608B7
:102F9000D8F80C100F6807F00303022B53D0032B53
:102FA00053D03F4A3F4F012B18BF1746D0F89040EF
:102FB0004FEA451E002205F1100C04EB0E03C3F886
:102FC000102B8A69002A42D04A8A05F158033A43F5
:102FD0005B01E2500123D4F81C2803FA0CF31343DD
:102FE000C4F81C38A64400234A69CEF8103905F10C
:102FF0003F03002A3BD00A8A04EB8303898B9208A3
:10300000012988BF4A43D0F89810561841EA024275
:103010002946C0F8986020465A60FFF775FED8F838
:103020000C301B8A43EA85531F4305F148035B01BB
:10303000E7500123D4F81C2803FA05F51543C4F81A
:103040001C58BDE8F081184FB0E7184FAEE704EB0D
:103050004613D3F8002B22F40042C3F8002B0123BF
:10306000D4F81C2803FA0CF322EA0303B8E704EBB4
:1030700083030F4A04EB461629465A602046FFF7A1
:1030800043FED6F80039012223F4004302FA05F585
:10309000C6F80039D4F81C3823EA0505CFE700BF8D
:1030A00000800010008004100080081000800C10C8
:1030B00000040002D0F894201268C0F89820FFF7AE
:1030C000B3BD00005831D0F8903049015B5813F47B
:1030D000004004D013F4001F14BF012002207047E9
:1030E0004831D0F8903049015B5813F4004004D0C7
:1030F00013F4001F14BF01200220704700EB810170
:10310000CB68196A0B6813604B6853607047000006
:1031100000EB810330B5DD68AA691368D36019B983
:10312000402B84BF402313606B8A1468D0F8902032
:103130001C4402EB4110013C09B2B4FBF3F46343BD
:10314000033323F0030343EAC44343F0C043C0F80E
:10315000103B2B6803F00303012B0ED1D2F8083883
:1031600002EB411013F4807FD0F8003B14BF43F012
:10317000805343F00053C0F8003B02EB4112D2F8F9
:10318000003B43F00443C2F8003B30BD2DE9F04161
:10319000D0F8906005460C4606EB4113D3F8087B47
:1031A0003A07C3F8087B08D5D6F814381B0704D5AE
:1031B00000EB8103DB685B689847FA072FD5D6F8E8
:1031C0001438DB072BD505EB8403D968CCB98B69A0
:1031D000488A5E68B6FBF0F200FB12628AB9186892
:1031E000DA6890420DD2121A83E81400202383F388
:1031F000118821462846FFF78BFF84F31188BDE82C
:10320000F081012303FA04F26B8923EA02036B8144
:10321000CB6823B121462846BDE8F0411847BDE8F8
:10322000F081000000EB81034A0170B5DD68D0F841
:1032300090306C692668E66056BB1A444FF4002053
:10324000C2F810092A6802F00302012A0AB20ED15C
:10325000D3F8080803EB421410F4807FD4F8000977
:1032600014BF40F0805040F00050C4F8000903EB58
:103270004212D2F8000940F00440C2F800090122CD
:10328000D3F8340802FA01F10143C3F8341870BDD1
:1032900019B9402E84BF4020206020681A442E8A2D
:1032A000841940F00050013CB4FBF6F440EAC440FD
:1032B000C6E700002DE9F041D0F8906004460D46C5
:1032C00006EB4113D3F80879C3F80879FB071CD53E
:1032D000D6F81038DA0718D500EB8103D3F80CE0E4
:1032E000DEF81430D3F800C0DA6894451BD2A2EBA4
:1032F0000C024FF000081A60C3F80480202383F307
:103300001188FFF78FFF88F311883B0618D501233A
:10331000D6F83428AB40134212D029462046BDE8E7
:10332000F041FFF7ADBC012303FA01F2038923EA60
:1033300002030381DEF80830002BE6D09847E4E76B
:10334000BDE8F0812DE9F047D0F8905004466E6951
:10335000AB691E40F1046E6103D5BDE8F047FEF78E
:1033600045BC002E12DAD5F8003E9A0705D0D5F8F4
:10337000003E23F00303C5F8003ED5F8043820468C
:1033800023F00103C5F80438FEF764FC330505D5C6
:103390002046FFF749FC2046FEF74CFCB7040CD54D
:1033A000D5F8083813F0060FEB6823F470530CBF00
:1033B00043F4105343F4A053EB60300704D5636823
:1033C000DB680BB120469847F10200F1A180B20200
:1033D0000BD5D4F8908000274FF00109D4F8943031
:1033E000F9B29B688B4280F0D280F3061AD5D4F8EC
:1033F00090100A6AC2F30A1702F00F0302F4F012E7
:10340000B2F5802F00F0EB80B2F5402F0AD104EB2B
:10341000830301F58051DB68186A00231A469F4236
:1034200040F0D1803003D5F8185835D5E90303D5DD
:1034300000212046FFF7AAFEAA0303D5012120465A
:10344000FFF7A4FE6B0303D502212046FFF79EFE83
:103450002F0303D503212046FFF798FEE80203D58A
:1034600004212046FFF792FEA90203D5052120463C
:10347000FFF78CFE6A0203D506212046FFF786FE81
:103480002B0203D507212046FFF780FEEF0103D56D
:1034900008212046FFF77AFE700340F1C780E90754
:1034A00003D500212046FFF705FFAA0703D5012118
:1034B0002046FFF7FFFE6B0703D502212046FFF7EA
:1034C000F9FE2F0703D503212046FFF7F3FEEE0692
:1034D00003D504212046FFF7EDFEA80603D50521FC
:1034E0002046FFF7E7FE690603D506212046FFF7D1
:1034F000E1FE2A0603D507212046FFF7DBFEEB0598
:1035000040F1948020460821BDE8F047FFF7D2BE85
:10351000D4F890904FF000084FF0010AD4F894309E
:103520005FFA88F79B68BB42FFF451AF09EB471382
:10353000D3F8002902F44022B2F5802F24D1D3F829
:103540000029002A20DAD3F8002942F09042C3F87B
:103550000029D3F80029002AFBDB3946D4F8900073
:10356000FFF7D2FB22890AFA07F322EA0303238139
:1035700004EB8703DB689B6813B139462046984704
:1035800039462046FFF77CFB08F10108C6E708EB47
:103590004112D2F8003B03F44023B3F5802F10D141
:1035A000D2F8003B002B0CDA628909FA01F322EA17
:1035B0000303638104EB8103DB68DB680BB1204606
:1035C000984701370AE713F0030F00D10A68072B69
:1035D00003F101039EBF0270120A01301FE704EBE2
:1035E000830301F58051DA6890690268D0F808C059
:1035F0004068A2EB000E00221046974208D1DB681B
:103600009B699A683A449A605A6817445F6009E770
:1036100012F0030F00D10868964502F1010282BF43
:103620008CF80000000A0CF1010CE6E7BDE8F08719
:1036300008B50348FFF786FEBDE80840FFF76ABA01
:103640002845002008B50348FFF77CFEBDE8084088
:10365000FFF760BAC4450020D0F8903003EB411169
:10366000D1F8003B43F40013C1F8003B7047000061
:10367000D0F8903003EB4111D1F8003943F4001336
:10368000C1F8003970470000D0F8903003EB4111C9
:10369000D1F8003B23F40013C1F8003B7047000051
:1036A000D0F8903003EB4111D1F8003923F4001326
:1036B000C1F800397047000000F1604300F01F02BC
:1036C0000901400903F56143C9B2800083F8001382
:1036D000012300F16040934000F56140C0F8803163
:1036E0000360704730B50433039C0172002104FB72
:1036F0000325C361049B00600363059B4060C160B8
:10370000426102618561046242628162C162436317
:1037100030BD00000022416AC260416101616FF06A
:1037200001018262C262FEF7E3BD000003694269E3
:10373000934203D1C2680AB100207047181D704738
:10374000036919600021C2680132C260C269134472
:1037500082699342036124BF436A0361FEF7BCBDE3
:1037600038B504460D46E3683BB162690020131D7D
:103770001268A3621344E36238BD237A33B9294641
:103780002046FEF799FD0028EDDA38BD6FF0010004
:10379000FBE70000C368C269013BC360436913448F
:1037A00082699342436124BF436A43610023836279
:1037B000036B03B11847704770B52023044683F3A9
:1037C0001188866A3EB9FFF7CBFF054618B186F32C
:1037D0001188284670BDA36AE26A13F8015B934220
:1037E000A36202D32046FFF7D5FF002383F311889D
:1037F000EFE700002DE9F84F04460E469046994643
:10380000202787F311880025AA46D4F828B0BBF1F9
:10381000000F09D149462046FFF7A2FF20B18BF3E4
:1038200011882846BDE8F88FA16AA8EB050BE36A6A
:103830005B1A9B4528BF9B46BBF1400F1BD9334603
:1038400001F1400251F8040B914243F8040BF9D105
:10385000A36A403640354033A362A26AE36A9A42C3
:1038600002D32046FFF796FF8AF311884545D8D248
:1038700087F31188C9E730465A46FDF783FBA36AF0
:103880005E445D445B44A362E7E7000010B5029C20
:1038900004330172C36103FB0421002300608362CF
:1038A000C362039B40600363049BC4604261026186
:1038B000816104624262436310BD0000026A6FF0DE
:1038C0000101C260426A4261026100228262C262F8
:1038D000FEF70EBD436902699A4203D1C2680AB17C
:1038E00000207047184650F8043B0B6070470000FA
:1038F000C3680021C2690133C3604369134482690C
:103900009342436124BF436A4361FEF7E5BC000074
:1039100038B504460D46E3683BB1236900201A1D03
:10392000A262E2691344E36238BD237A33B92946BF
:103930002046FEF7C1FC0028EDDA38BD6FF001002B
:10394000FBE7000003691960C268013AC260C269FE
:10395000134482699342036124BF436A03610023D5
:103960008362036B03B118477047000070B52023D2
:1039700004460E4683F31188856A35B91146FFF770
:10398000C7FF10B185F3118870BDA36A1E70A36ACA
:10399000E26A01339342A36204D3E1692046043909
:1039A000FFF7D0FF002080F3118870BD2DE9F84F9C
:1039B00004460D4691469A464FF0200888F3118838
:1039C0000026B346A76A4FB951462046FFF7A0FF2D
:1039D00020B187F311883046BDE8F88FA06AA9EBC3
:1039E0000603E76A3F1A9F4228BF1F46402F1BD994
:1039F00005F1400355F8042B9D4240F8042BF9D102
:103A0000A36A40364033A362A26AE36A9A4204D3AF
:103A1000E16920460439FFF795FF8BF311884E4585
:103A2000D9D288F31188CDE729463A46FDF7AAFA9C
:103A3000A36A3D443E443B44A362E5E7026943690F
:103A40009A4203D1C3681BB9184670470023FBE7AD
:103A5000836A002BF8D0043B9B1AF5D01360C3682F
:103A6000013BC360C3691A4483699A42026124BF5F
:103A7000436A0361002383620123E5E700F0D0B8C5
:103A80004FF08043002258631A610222DA607047C7
:103A900000224FF08043DA60704700004FF080430F
:103AA000586370474FF08043586A70474B684360D3
:103AB0008B688360CB68C3600B6943614B690362A9
:103AC0008B6943620B6803607047000008B5304B98
:103AD00040F2FF712F48D3F888200A43C3F88820AA
:103AE000D3F8882022F4FF6222F00702C3F888206E
:103AF000D3F88820D3F8E0200A43C3F8E020D3F8B5
:103B000008210A43C3F80821234AD3F80831114693
:103B1000FFF7CCFF214802F11C01FFF7C7FF204847
:103B200002F13801FFF7C2FF1E4802F15401FFF70E
:103B3000BDFF1D4802F17001FFF7B8FF1B4802F1FD
:103B40008C01FFF7B3FF1A4802F1A801FFF7AEFF9F
:103B5000184802F1C401FFF7A9FF174802F1E0017C
:103B6000FFF7A4FF154802F1FC01FFF79FFF14487F
:103B700002F58C71FFF79AFF00F004F9114B052252
:103B80009A604FF06052DA600F4A1A6108BD00BFB8
:103B90000044025800000258D443000800040258B0
:103BA00000080258000C0258001002580014025875
:103BB00000180258001C0258002002580024025825
:103BC0000028025890ED00E01F00080308B500F03F
:103BD000D5FAFEF7F9FA0F4BD3F8DC2042F0400299
:103BE000C3F8DC20D3F8042122F04002C3F80421FA
:103BF000D3F80431084B1A6842F008021A601A68B8
:103C000042F004021A60FEF739FFBDE80840FEF7F3
:103C1000E9BC00BF00440258001802487047000089
:103C2000114BD3F8E82042F00102C3F8E820D3F8A2
:103C3000102142F00102C3F810210C4AD3F81031D0
:103C4000D36B43F00103D3634FF08043C7229A62E2
:103C50004FF0FF32DA6200229A615A63DA605A60EA
:103C600001225A611A607047004402580010005C3B
:103C70004FF0804208B51369D1680B40D9B29B0759
:103C80006FEA0101116107D5202383F31188FEF744
:103C9000BBFA002383F3118808BD0000384B4FF0B6
:103CA000FF31D3F88020C3F88010D3F880200022A1
:103CB000C3F88020D3F88000D3F88400C3F88410C0
:103CC000D3F88400C3F88420D3F88400D86F40F080
:103CD000FF4040F4FF0040F43F5040F03F00D86701
:103CE000D86F20F0FF4020F4FF0020F43F5020F078
:103CF0003F00D867D86FD3F888006FEA40506FEA6A
:103D00005050C3F88800D3F88800C0F30A00C3F805
:103D10008800D3F88800D3F89000C3F89010D3F847
:103D20009000C3F89020D3F89000D3F89400C3F823
:103D30009410D3F89400C3F89420D3F89400D3F8E7
:103D40009800C3F89810D3F89800C3F89820D3F8D7
:103D50009800D3F88C00C3F88C10D3F88C00C3F80B
:103D60008C20D3F88C00D3F89C00C3F89C10D3F8B7
:103D70009C10C3F89C20D3F89C3000F0D3B900BF4E
:103D8000004402580122614B1A60614BD3F8F420C1
:103D900042F00202C3F8F420D3F81C2142F00202E0
:103DA000C3F81C210222D3F81C315A4BDA605A683E
:103DB0009104FCD5584A1A6001229A60574ADA6089
:103DC00000221A614FF440429A61524B9A69920460
:103DD000FCD51A6842F480721A604D4B1A6F12F4C7
:103DE000407F04D04FF480321A6700221A671A68A5
:103DF00042F001021A60464A134611684807FCD592
:103E0000002111611A6912F03802FBD101211960F9
:103E10004FF0804159605A67414ADA62414A1A615B
:103E20001A6842F480321A60394A134611688903CD
:103E3000FCD5116841F4805111601A689204FCD5D8
:103E4000394A3A499A6200225A6319633849DA6357
:103E500099635A64374A1A64374ADA621A6842F038
:103E6000A8521A602A4B1A6802F02852B2F1285F51
:103E7000F9D148229A614FF48862DA6140221A62CD
:103E80002E4ADA644FF000521A652D4A5A652D4ABF
:103E90009A6532222C4B1A601A6802F00F02022A2D
:103EA000FAD11B4B1A6942F003021A611A6902F037
:103EB0003802182AFAD1D3F8DC2042F00052C3F8B5
:103EC000DC20D3F8042142F00052C3F80421D3F8D7
:103ED0000421D3F8DC2042F08042C3F8DC20D3F880
:103EE000042142F08042C3F80421D3F80421D3F81E
:103EF000DC2042F00042C3F8DC20D3F8042142F079
:103F00000042C3F80421D3F80431704708810051FE
:103F1000004402580048025800C000F002000001AE
:103F20000000FF01008890081210200063020701C2
:103F30002C02040047040508FD0BFF0120000020AF
:103F40000010E00000010100002000524FF0B042DC
:103F500008B5D2F8883003F00103C2F8883023B1E5
:103F6000044A13680BB150689847BDE80840FEF753
:103F7000D1BD00BF784600204FF0B04208B5D2F85E
:103F8000883003F00203C2F8883023B1044A9368F2
:103F90000BB1D0689847BDE80840FEF7BBBD00BF35
:103FA000784600204FF0B04208B5D2F8883003F0D0
:103FB0000403C2F8883023B1044A13690BB1506975
:103FC0009847BDE80840FEF7A5BD00BF7846002031
:103FD0004FF0B04208B5D2F8883003F00803C2F8B9
:103FE000883023B1044A93690BB1D0699847BDE882
:103FF0000840FEF78FBD00BF784600204FF0B0426A
:1040000008B5D2F8883003F01003C2F8883023B125
:10401000044A136A0BB1506A9847BDE80840FEF79E
:1040200079BD00BF784600204FF0B04310B5D3F8FB
:10403000884004F47872C3F88820A30604D5124A95
:10404000936A0BB1D06A9847600604D50E4A136B89
:104050000BB1506B9847210604D50B4A936B0BB1FB
:10406000D06B9847E20504D5074A136C0BB1506C2E
:104070009847A30504D5044A936C0BB1D06C9847BC
:10408000BDE81040FEF746BD784600204FF0B04333
:1040900010B5D3F8884004F47C42C3F88820620548
:1040A00004D5164A136D0BB1506D9847230504D5FE
:1040B000124A936D0BB1D06D9847E00404D50F4AB6
:1040C000136E0BB1506E9847A10404D50B4A936E42
:1040D0000BB1D06E9847620404D5084A136F0BB138
:1040E000506F9847230404D5044A936F0BB1D06FE7
:1040F0009847BDE81040FEF70DBD00BF7846002090
:1041000008B50348FDF700F9BDE80840FEF702BD19
:10411000CC23002008B5FFF7ABFDBDE80840FEF753
:10412000F9BC0000062108B50846FFF7C5FA0621CC
:104130000720FFF7C1FA06210820FFF7BDFA062184
:104140000920FFF7B9FA06210A20FFF7B5FA062180
:104150001720FFF7B1FA06212820FFF7ADFA092151
:104160007A20FFF7A9FA07211C20FFF7A5FA0C21F6
:104170005220BDE80840FFF79FBA000008B5FFF7DE
:104180008DFD00F00DF8FDF7D9FAFDF7B3FCFDF752
:1041900083FBFFF743FDBDE80840FFF76FBC00005D
:1041A000002304491A465A50C81808334260802B2D
:1041B000F9D1704778460020121012131211000036
:1041C000F0290020CC23002053544D333248373F90
:1041D0003F3F0053544D3332483734332F37353354
:1041E0000000000000960000000000000000000039
:1041F00000000000000000000000000000000000BF
:1042000005170008F11600082D17000819170008F7
:104210002517000811170008FD160008E916000808
:10422000391700080000000011180008FD170008E9
:104230003918000825180008311800081D18000852
:1042400009180008F517000895180008000000007C
:1042500001000000000000006D61696E00000000B8
:104260007842000878280020F02900200100000092
:10427000C52100080000000069646C6500000000B2
:1042800002000000000000003D1A0008A91A000802
:104290004000400098420020A84200200200000098
:1042A000000000000300000000000000F11A0008F8
:1042B0000000000010000000B842002000000000D4
:1042C000010000000000000028450020010102005C
:1042D0004172647550696C6F740025424F415244BD
:1042E000252D424C002553455249414C25000000E4
:1042F000852500089D24000835250008192500089B
:10430000430000000843000809024300020100C006
:104310003209040000010202010005240010010519
:10432000240100010424020205240600010705827D
:10433000030800FF09040100020A0000000705014C
:10434000024000000705810240000000120000004A
:1043500054430008120110010200004009124157A5
:1043600000020102030100000403090425424F4139
:104370005244250051696F54656B5A65616C6F74C6
:1043800048373433003031323334353637383941F9
:10439000424344454600000000000000691C00083C
:1043A000491F0008F51F000840004000604600203B
:1043B00060460020010000007046002080000000E0
:1043C000400100000800000000010000000400009F
:1043D000080000000000916A00000000AAAAAAAA32
:1043E00000001140FFFF00000000000000A00A00D4
:1043F0001000000000000000AAAAAAAA10000000F5
:10440000FFFF00000000000000000000000010009E
:1044100000000000AAAAAAAA00001000FFFF0000E6
:10442000000000000000000000400000000000004C
:10443000AAAAAAAA00400000FFFF00000000000096
:10444000000000005580120107000000AAAAAAAAD5
:1044500040401101FFFF0000000000700700000055
:104460000000000000000000AAAAAAAA00000000A4
:10447000FFFF00000000000000000000000000003E
:1044800000000000AAAAAAAA00000000FFFF000086
:10449000000000000000000000000000000000001C
:1044A000AAAAAAAA00000000FFFF00000000000066
:1044B000000000000000000000000000AAAAAAAA54
:1044C00000000000FFFF00000000000000000000EE
:1044D0000000000000000000AAAAAAAA0000000034
:1044E000FFFF0000000000000000000000000000CE
:1044F00000000000AAAAAAAA00000000FFFF000016
:1045000000000000000000000C040000000000009B
:1045100000001E0000000000FF000000000000007E
:10452000C84100083F00000050040000D3410008CB
:104530003F00000000960000000008009600000008
:1045400000080000040000006843000800000000AC
:10455000000000000000000000000000000000005B
:044560000000000057
:00000001FF
